:100000000C94EB000C9457090C9408010C94080113
:100010000C9408010C9408010C9408010C9408013C
:100020000C9408010C9408010C9408010C9408012C
:100030000C9408010C9408010C9408010C9408011C
:100040000C9408010C9408010C9408010C9408010C
:100050000C94080143066B06A3065009CA06DE0687
:100060004C07500950094F075009500950095009D1
:1000700050095507600780079207CA076308A1085F
:100080000F092409550848083109D106490900001B
:10009000000000000000020006000E001200140024
:1000A0001500170018001A001B001D001E0020007C
:1000B000210024002600270029002C002D003000FC
:1000C0003200350038003B003E004100440047004C
:1000D0004B004E00530057005C0060006500690053
:1000E0006F0074007A00800087008D0095009C00EE
:1000F000A400AB00B400BD00C600D100DA00E600E9
:10010000F000FC00080116012301320141015201F7
:100110006201730186019801AD01C201D901EF01AD
:10012000090222023D025A0276029602B702D90261
:10013000FB0223034A0374039F03CC03FC032D0437
:1001400062049904D404110550059405DA052306C8
:100150007006C10616077007CE0730089608030917
:100160007309EB09680AEB0A720B020C9D0C3B0D3C
:10017000DE0D910E470F0810CB10A01181126D13E8
:100180005614561560168617A318DC191E1B811C01
:10019000EC1D5E1FD1208F222924EA25DA27C529EC
:1001A000E12BF22D3730B9322335CB374B3A073DAF
:1001B000074057436046654A1E4EE251F055345A97
:1001C000935E42632868426D8B722F78347E688418
:1001D000C18ABF91E09811241FBECFE5D8E0DEBFF1
:1001E000CDBF10E0A0E6B0E0E2E2F8E202C0059088
:1001F0000D92A039B107D9F712E0A0E9B0E001C033
:100200001D92AA32B107E1F70E9464050C940F1405
:100210000C94000087B38E7587BB18BA089588B315
:100220008E7188BBBE9887B3816A87BB0895E82F1B
:100230008091BF009091C000079728F4EFB9779B99
:10024000FECF7FB126C02091B5003091B600369523
:10025000279560E870E040E050E0862F8E2311F093
:10026000C59A01C0C598C9010197F1F7C79AC9019C
:100270000197F1F7B699762BC9010197F1F7C79865
:10028000C9010197F1F766954F5F5F4F48305105FF
:1002900021F7872F08958DB19EB11DB81EB820910A
:1002A000B5003091B600F9013197F1F7C79AF9011D
:1002B0003197F1F7C7988DB99EB90895FF920F93C2
:1002C0001F93162F072FF42E0E941701802F0E94D4
:1002D0001701812F0E9417018F2D0E9417011F9176
:1002E0000F91FF9008950E941701089580E00E94E9
:1002F000170108951F931FB7F8948091BD00909146
:10030000BE00019749F48BE267E00E94E70C10926F
:10031000BE001092BD000AC08BE263E00E94E70CB1
:1003200081E090E09093BE008093BD001FBF1F91BD
:100330000895FC018181813011F40E94AF1208956B
:100340000F931F93182F0FB7F8948BE268E00E9469
:10035000E70C89E267EC70E0412F0E94C50C0E9417
:100360007A010FBF1F910F910895CF92DF92EF9204
:10037000FF920F931F93CF93DF938C01FC01818138
:100380008D3348F482818D3330F46801EE24FF24EC
:10039000C0E0D0E01EC08DE18093C70089EC80935F
:1003A000C80082E02FC0F60184810E941701282F27
:1003B000F801838190E0E816F9062CF0FE01E9537C
:1003C000FF4F228321960894E11CF11C0894C11C64
:1003D000D11CF801818190E0E816F90624F38281AE
:1003E00090E0C817D90714F480E0DFCF8DE1809347
:1003F000C7001092C800FE01E953FF4F12829E0110
:100400002D5F822F0E94A001DF91CF911F910F914C
:10041000FF90EF90DF90CF900895CF92DF92EF9210
:10042000FF920F931F93CF93DF93EC011092A700DD
:100430001092A8001092A9001092AA001092AF008A
:100440008FEF9FEF9093B4008093B3008091B20040
:100450008B7F8093B2008091B2008E7F8093B20038
:100460000E940F01DC9AC7988091C5009091C60048
:10047000019761F4C0988AE090E00E94B712C09A98
:100480008AE090E00E94B712C0980BC0C09A8AE040
:1004900090E00E94B712C0988AE090E00E94B712E4
:1004A000C09A8AE090E00E94B71280E18093C70072
:1004B0008B8190E00E94B7128C8100E010E0C82E82
:1004C000DD2433C088850E9417018D8190E00E9451
:1004D000B71289850E9417018D8190E00E94B712A2
:1004E0008A850E941701E82E8D8190E00E94B71244
:1004F0008B850E941701F82E8D8190E00E94B71223
:100500008F81882359F0833021F48E81E81649F4D5
:1005100005C0843031F48E81F81619F41092C800A9
:100520000AC00E944B010F5F1F4FC016D10651F643
:1005300080EC8093C80082E00E94A001DF91CF91FF
:100540001F910F91FF90EF90DF90CF9008956F92E1
:100550007F928F929F92AF92BF92CF92DF92EF9253
:10056000FF920F931F93CF93DF93EC016B01B42E97
:100570008091C800882309F068C1442319F0A09035
:10058000A60002C0A090A500EE24FF2400E0F8EE33
:100590008F2EF3E09F2EE1E87E2E70E8672EE1C0FB
:1005A0008091B20082FF2DC02091A7003091A80059
:1005B0004091A9005091AA008091B3009091B4009D
:1005C0009A0144275527A0E0B0E0281739074A07C9
:1005D0005B07B9F08091A7009091A800A091A900B5
:1005E000B091AA00CD01AA27BB279093B4008093B5
:1005F000B3006091B3007091B4008DE440E00E94BC
:100600005E01BB2059F4E0FE04C08091A200886026
:1006100003C08091A200877F8093A2008091A200F6
:100620002091A7003091A8004091A9005091AA0004
:10063000B90148810E945E018091A00080FD50C0F8
:100640001091A100110F110F8091A00083FF17C01E
:10065000C4010197F1F780EF60E070E040E00E9494
:100660005E0190E09C012170307080FF02C011504B
:1006700079F7232B09F455C07092AF0052C08091D6
:10068000A00082FF27C088818A1521F1BB2059F480
:10069000E0FE04C08091A400886003C08091A400A3
:1006A000877F8093A400C4010197F1F78091A40093
:1006B0002091A7003091A8004091A9005091AA0074
:1006C000B90140E00E945E019881891751F11150F3
:1006D00051F7D4C08091A10090E00E94B71221C0D0
:1006E00088818A15F1F08091B20080FD1AC0809156
:1006F000A7009091A800A091A900B091AA009093A2
:10070000B1008093B000902F9170990F8091B2004A
:100710008D7F892B8093B2008091B200816080939D
:10072000B200BB2011F4E0FE13C08091A7009091AD
:10073000A800A091A900B091AA000196A11DB11D29
:100740008093A7009093A800A093A900B093AA005B
:100750000894C108D1080894E11CF11C21960F5F90
:100760000170C114D10409F01BCF8091A0008178E1
:10077000813809F05FC01091A100110F110F809115
:10078000A3002091AB003091AC004091AD0050919E
:10079000AE00B90140E00E945E018091A00086FF9A
:1007A00017C0C8EED3E0CE010197F1F780EF60E00B
:1007B00070E040E00E945E0190E09C01217030708A
:1007C00080FF02C0115079F7232BA1F181E82AC0E4
:1007D0008091A00085FF29C08091B20080FF25C0D4
:1007E000BB2069F48091B20081FF04C08091A40015
:1007F000886003C08091A400877F8093A400C8EE26
:10080000D3E0CE010197F1F78091A4006091B00090
:100810007091B10040E00E945E018A1559F41150B8
:1008200081F780E88093AF0005C08091A10090E03F
:100830000E94B712BB2011F483E101C085E18093CF
:10084000C7008091AF008093C8001092AF008091E4
:10085000B2008E7F8093B20082E00E94A001DF91FF
:10086000CF911F910F91FF90EF90DF90CF90BF90AD
:10087000AF909F908F907F906F9008956092AF009F
:1008800050CF80919E0090919F00892B09F44CC01D
:100890008BE268E00E94E70C80919E0090919F009F
:1008A0008134910528F16091C1007091C200B6E0D9
:1008B000660F771FBA95E1F769537F4F89E240E4ED
:1008C0000E94C50C8091C1009091C2000196909346
:1008D000C2008093C10080919E0090919F0080543F
:1008E000904090939F0080939E000E947A0108950B
:1008F0006091C1007091C20040919E0050919F0094
:10090000A6E0660F771FAA95E1F769537F4F89E24A
:100910000E94C50C1092C2001092C10010929F005C
:1009200010929E000E947A0108950F931F93AC01CC
:100930008091BB009091BC00892B11F400E41CC095
:10094000465F5F4F8091B8008093C7006093B70007
:1009500087EE90E0909391008093900080919E00AC
:1009600090919F008D50914020F080EC8093C800C2
:1009700002C01092C80006E380919E0090919F00F3
:10098000202F30E02817390788F480919E0090913D
:100990009F00821B930B90939F0080939E0081E0A9
:1009A00090E09093BA008093B9000DC080919E00B2
:1009B00090919F00082F10929F0010929E0010921D
:1009C000BA001092B9008091C8008823A1F410E009
:1009D0008091900090919100BA01402F50E00E94C8
:1009E000F1138091900090919100800F911F90934E
:1009F00091008093900080919E0090919F00892BA0
:100A000019F481E0809315021F910F91089580E001
:100A100090E00E94FA1390E09093C0008093BF0092
:100A20008091BF009091C000843A910530F083E03E
:100A300090E09093C0008093BF0088B38F7188BB13
:100A4000BE9821EA27BBBC9A1DB81EB8E091BF0032
:100A5000F091C000EE0FFF1FE257FF4F8591949178
:100A60009093B6008093B5008091BF009091C00034
:100A700083309105C1F08430910530F481309105C7
:100A800071F0029770F409C08530910599F08530B6
:100A9000910558F00697A1F40FC080E507C083E5E3
:100AA00005C081E503C081E508C082E58DB981E01C
:100AB0008EB9089582E501C083E58DB91EB8089509
:100AC000C798BE9827BB08956F927F928F929F928E
:100AD000AF92BF92CF92DF92EF92FF920F93DF938C
:100AE000CF9300D0CDB7DEB70E94070587B38E75D0
:100AF00087BB18BA0E94F80C1092BA001092B90085
:100B000081E090E09093C4008093C3001092C200F3
:100B10001092C1009093C6008093C5001092BE0051
:100B20001092BD0010929100109290001092150248
:100B300080E18ABBDC98C09A8BEE93E00E944F0D57
:100B400084E091E20E94540D80E092E00E94590DF1
:100B500089E0898384E08A83CE0101960E942D1169
:100B600080E690E00E94CB1189E690E00E94C311DC
:100B70008AE790E00E94BB110E9403114C0162E3DE
:100B800070E00E94670DC40160E070E00E9479107F
:100B90003C01C401B30140E050E00E948D0DC4014E
:100BA000B30141E050E022E030E002E0A0E4EA2EB0
:100BB000F12CCC24DD24F1E4AF2EF4E0BF2E0E9412
:100BC0002710C401B30141E050E022E030E0E5E04D
:100BD000AE2EE6E0BE2E0E9451100E94790C789451
:100BE0000E94FA11809115028823E1F36091900030
:100BF00070919100675E7040109215024091B700AD
:100C000087EE90E00E94A702EDCFEF92FF920F9344
:100C10001F93CF93DF93182FEB018BE260E00E94CC
:100C2000E70C8BE268E00E94E70C112309F438C35B
:100C30008091B9009091BA00892B91F08091B80011
:100C4000833121F4CE0160E00E9495048091B800C8
:100C5000853109F025C3CE0161E00E94950420C3CF
:100C600088818093B800888190E0FC013197ED3154
:100C7000F10508F015C3E65DFF4FEE0FFF1F05906D
:100C8000F491E02D099481E08093C7001092C80090
:100C90008AE08093C90081E48093CA0086E580934E
:100CA000CB0082E58093CC0089E48093CD0083E57E
:100CB0008093CE0080E58093CF008FE58093D000B5
:100CC0008DE48093D1008BE48093D20082E3809303
:100CD000D3008DE0DBC282E08093C7001092C80091
:100CE0008981883991F08E3909F059C08A81882329
:100CF00029F41092C6001092C50051C081E090E026
:100D00009093C6008093C5004AC08A81843A10F04F
:100D100083EA8A838A81682F70E08091BF00909176
:100D2000C0006817790761F07093C0006093BF003E
:100D30006091BF007091C00080E090E00E940214BA
:100D40000E9407052CC083E08093C7001092C80062
:100D500069816239A1F0633938F4603909F470C2ED
:100D6000613909F06DC209C0683969F0613A09F466
:100D700067C2643909F064C204C082E008C08AE036
:100D800006C082E304C08091BF009091C0008093B0
:100D9000C90058C285E08093C7001092C80082E065
:100DA00075C28A810E9417018B810E9417018C8174
:100DB0000E9417010E9476019CE15FC2898190E048
:100DC000A0E0B0E08093A7009093A800A093A900B2
:100DD000B093AA002091A7003091A8004091A900EB
:100DE0005091AA008A8190E0A0E0B0E0542F432FF8
:100DF000322F2227822B932BA42BB52B8093A70075
:100E00009093A800A093A900B093AA002091A700F6
:100E10003091A8004091A9005091AA008B8190E0E8
:100E2000A0E0B0E0542F432F322F2227822B932BA8
:100E3000A42BB52B8093A7009093A800A093A900A2
:100E4000B093AA002091A7003091A8004091A9007A
:100E50005091AA008C8190E0A0E0B0E0542F432F85
:100E6000322F2227822B932BA42BB52B8093A70004
:100E70009093A800A093A900B093AA0020E08981D4
:100E800087FD21E0220F220F8091B2008B7F822B01
:100E90008093B20086E07FCF0E94AF1201C28AE049
:100EA0008093C7001092C800FBC1CE010E940D02C2
:100EB0008091B2008E7F8093B2001092AF00F0C19B
:100EC0008DE460E070E040E00E945E01DC98C09A32
:100ED00087B38E7587BB18BA81E18093C7001092E3
:100EE000C80082E00E94A0018091C3009091C400DC
:100EF000892B09F0D5C11092BE001092BD00D0C15F
:100F00008B810E9417018C810E94170180E00E9452
:100F1000170180E00E941701898190E00E94B712BA
:100F200082E139CF998180E02A8130E0822B932BB6
:100F300090939F0080939E008B818093A0008C8172
:100F40008093A1008D818093A2008E818093A30065
:100F50008F818093A40088858093A50089858093E4
:100F6000A6008091A7009091A800A091A900B0913F
:100F7000AA008093AB009093AC00A093AD00B09317
:100F8000AE0081E090E09093BC008093BB00CE0166
:100F900060E0D0C0998180E02A8130E0822B932BE1
:100FA000019690939F0080939E008B818093A40074
:100FB00000919E0010919F00C9ECD0E008531F4F94
:100FC000E0E2EE2E78E2F72E5DC08091B20082FF63
:100FD0002DC02091A7003091A8004091A900509108
:100FE000AA008091B3009091B4009A01442755273C
:100FF000A0E0B0E0281739074A075B07B9F08091F5
:10100000A7009091A800A091A900B091AA00CD01DD
:10101000AA27BB279093B4008093B3006091B300DC
:101020007091B4008DE440E00E945E018091A400C4
:101030002091A7003091A8004091A9005091AA00EA
:10104000B90140E00E945E0188838091A400803253
:1010500019F4F092A40015C0E092A4008091A700BA
:101060009091A800A091A900B091AA000196A11D9D
:10107000B11D8093A7009093A800A093A900B093FE
:10108000AA002196C017D10709F09FCF84E197C02D
:101090008A810E9417018B810E9417018C810E9416
:1010A00017010E9476019AE1E8C089810E94170128
:1010B0008A810E9417018B810E9417018C810E94F6
:1010C000170189E1B9C0998180E02A8130E0822B43
:1010D000932B90939F0080939E008B818093A00020
:1010E0008C818093A1008D818093A2008E8180935A
:1010F000A3008F818093A40088858093A5008985B3
:101100008093A6008091A7009091A800A091A900CB
:10111000B091AA008093AB009093AC00A093AD0077
:10112000B093AE0081E090E09093BC008093BB0050
:10113000CE0161E00E9495041092BC001092BB00A9
:10114000AFC0998180E02A8130E0822B932B0196F9
:1011500090939F0080939E008B818093A4000091C8
:101160009E0010919F00C7ECD0E00C0F1D1F22C005
:101170008091A4002091A7003091A8004091A9007F
:101180005091AA00B90140E00E945E0189838091DC
:10119000A7009091A800A091A900B091AA00019683
:1011A000A11DB11D8093A7009093A800A093A90052
:1011B000B093AA002196C017D107D1F686E180939B
:1011C000C7001092C800E0919E00F0919F00E95383
:1011D000FF4F118280919E0090919F00CF9798F0D1
:1011E00080E40E94A00180919E0090919F00CE9784
:1011F00090939F0080939E0081E090E09093C200C6
:101200008093C1004DC080919E0090919F008E5FA1
:101210000E94A00110929F0010929E0041C08981FF
:101220000E9417018A810E9417018B810E94170179
:101230008C810E94170187E18093C7001092C8003B
:101240001092C90083E022C08A810E9417018B811D
:101250000E9417018C810E9417010E94760198E17B
:101260000CC08A810E9417018B810E9417018C811A
:101270000E9417010E9476019BE19093C700109293
:10128000C8008093C9001092CA0084E00E94A001A7
:1012900007C01092C4001092C300CE010E94B50195
:1012A000DF91CF911F910F91FF90EF9008951F92C2
:1012B0000F920FB60F9211242F933F934F935F938A
:1012C0006F937F938F939F93AF93BF93EF93FF930E
:1012D0000E94D311FF91EF91BF91AF919F918F9198
:1012E0007F916F915F914F913F912F910F900FBE22
:1012F0000F901F90189583E28093190281E28093EA
:10130000180280E280931A0210921B0288E090E09B
:1013100090931D0280931C0208950895089581E220
:10132000609125020E94E70C08958BE268E00E941C
:10133000E70C88E262E10E94E70C8FE268E00E941D
:10134000E70C8CE262E10E94E70C8FE261E00E9410
:10135000E70C83E265E00E94E70C08950F931F936A
:101360008C0180E260E40E94E70CF8016281605821
:1013700084E00E94E70CF8018281809324021F918F
:101380000F9108950F931F93CF93DF93EC0128855E
:101390003985121613060CF044C08E819F81821786
:1013A000930764F583E268E00E94E70C8E819F81D9
:1013B00008851985081B190B6A857B85083011057E
:1013C0005CF4680F791F81E2402F0E94C50C8E816A
:1013D0009F81800F911F09C0680F791F81E248E04B
:1013E0000E94C50C8E819F8108969F838E832885DD
:1013F00039858E819F818217930724F087E261E00F
:101400000E94E70C8B81813031F4898165E00E9474
:10141000E70C1B8206C0898161E00E94E70C81E035
:101420008B83DF91CF911F910F910895DF93CF931D
:1014300000D000D0CDB7DEB7FC01328123811092FD
:101440001F0210921E0281E080931B02223031F1B4
:101450002330B9F1213009F05FC0809103028093FD
:1014600020021092210283E092E090932302809365
:10147000220286819781089721F480E490E0978387
:101480008683868197818034910509F045C088E084
:1014900090E090932102809320023EC08681978144
:1014A0009093210280932002832F90E0880F991F50
:1014B000E0911602F0911702E80FF91F80819181E7
:1014C00027C03323B9F0832F90E0880F991FE09154
:1014D0009C00F0919D00E80FF91F0190F081E02D34
:1014E000F0932302E09322028081809320021092E5
:1014F000210212C094E099832A8389E08B839C8324
:1015000084E090E09093210280932002CE01019626
:10151000909323028093220288E192E00E94C20904
:101520000F900F900F900F90CF91DF910895CF9370
:10153000DF9382E20E94B50CC82F85FF1AC083E2B8
:1015400068E00E94E70CC6FF10C020911E02309197
:101550001F028091200290912102281739072CF454
:1015600088E192E00E94C20904C087E261E00E9423
:10157000E70CDF91CF9108950F931F9388E00E94AD
:10158000B50C082F182F86FF18C085E060E00E9478
:10159000E70C84E060E80E94E70C80E260E00E94D3
:1015A000E70C83E268E00E94E70C87E261E00E94BA
:1015B000E70C85E062E00E94E70C14FF04C089E0BC
:1015C00060EC0E94E70C07FF04C089E060ED0E9418
:1015D000E70C1F910F910895CF93DF938AE00E944B
:1015E000B50CC82F80FF02C00E94970AC1FF0AC035
:1015F0008AE20E94B50CE091F301F091F40130977A
:1016000009F00995C2FF0AC082E30E94B50CE0917F
:10161000F501F091F601309709F00995C3FF0AC072
:101620008AE30E94B50CE091F701F091F801309740
:1016300009F00995DF91CF9108958EE00E94B50CD5
:101640000895EF92FF920F931F93CF93DF93E82EAD
:10165000F62EEA0100E008C08F2DBE01412F0E9446
:10166000900C010FC10FD11D8E2D0E94B50C182FAB
:101670001F7091F7802FDF91CF911F910F91FF90F5
:10168000EF9008950F931F93DF93CF93CDB7DEB7FD
:1016900028970FB6F894DEBF0FBECDBF86E20E943A
:1016A000B50C86FF72C085E28E010F5F1F4FB80137
:1016B00048E00E94900C87E268E00E94E70C83E219
:1016C00068E00E94E70C80E20E94B50C682F6F77FB
:1016D00080E20E94E70C898190E0807690708032F1
:1016E000910509F440C080349105D1F1892BF1F5C1
:1016F000F80181818630D9F0873048F48130F1F1EA
:101700008130C8F0833079F1853081F521C089308E
:1017100019F18A3018F4883049F505C08A3071F122
:101720008B3021F520C081E26091250225C0C801DF
:101730000E94160A23C083E268E00E94E70C81E25F
:1017400061E00E94E70C81E260E00E94E70C0BC0C0
:10175000C8010E94AE0912C0C8010E9495090EC0BE
:10176000C8010E94990183E265E006C080E20E9400
:10177000B50C682F605880E20E94E70CF801808168
:101780008823D1F483E265E015C0209120023091D6
:10179000210280911C0290911D028217930764F42C
:1017A000109221021092200283E268E00E94E70C6E
:1017B00087E261E00E94E70C28960FB6F894DEBF3E
:1017C0000FBECDBFCF91DF911F910F910895EF9282
:1017D000FF920F931F93DF93CF93CDB7DEB7C05423
:1017E000D0400FB6F894DEBF0FBECDBFFE013196DC
:1017F00080E4DF011D928A95E9F78CE00E94B50C28
:10180000E82E80FF02C00E94420BE1FE20C08091C2
:10181000920090919300892B79F08EE26DE28E0117
:101820000F5F1F4FA8010E94210BE0919200F091E1
:101830009300B801099503C08EE20E94B50C8FE2B7
:1018400068E00E94E70C8FE261E00E94E70CE2FE94
:1018500020C08091940090919500892B79F086E3C7
:1018600065E38E010F5F1F4FA8010E94210BE091DD
:101870009400F0919500B801099503C086E30E9499
:10188000B50C87E368E00E94E70C87E361E00E9403
:10189000E70CE3FE20C08091960090919700892B81
:1018A00079F08EE36DE38E010F5F1F4FA8010E9458
:1018B000210BE0919600F0919700B801099503C0C3
:1018C0008EE30E94B50C8FE368E00E94E70C8FE383
:1018D00061E00E94E70CC05CDF4F0FB6F894DEBFFA
:1018E0000FBECDBFCF91DF911F910F91FF90EF9071
:1018F00008959FB7F89485B78E7F85BF85B78260BE
:1019000085BF8BB780648BBF8A9881B3886781BBA2
:1019100082B38B7B82BB82B3886382BB9FBF0895F7
:10192000FB019FB7F89485BB8FEF84BB969A939881
:101930009598959A939A969814BA00000000000022
:10194000000000000EC0939894980000000083B33C
:101950008193949A939A0000000000000000000018
:101960004150442381F79FBF0895DF93CF930F9297
:10197000CDB7DEB7BE016F5F7F4F41E00E94900C94
:1019800089810F90CF91DF910895FB019FB7F89463
:1019900085BB8FEF84BB969A93989598959A939A66
:1019A0009698000000000000000000000CC081912B
:1019B00085BB93989598959A939A00000000000033
:1019C000000000004150442391F79FBF0895DF932A
:1019D000CF930F92CDB7DEB76983BE016F5F7F4FA4
:1019E00041E00E94C50C0F90CF91DF9108950895BA
:1019F00082E18093030281E08093040280E191E020
:101A0000909306028093050210920702109208023A
:101A10001092090288E080930A0210920C02109240
:101A20000B0210920E0210920D02109210021092F0
:101A30000F021092110210921202109213021092D1
:101A4000140210929300109292001092950010923E
:101A5000940010929700109296001092F401109248
:101A6000F3011092F6011092F5011092F801109214
:101A7000F7011092FA011092F90110929B00109256
:101A80009A00089590930C0280930B0270930E02BB
:101A900060930D025093100240930F0208959093AB
:101AA0000C0280930B02089590930E0280930D0216
:101AB00008959093100280930F0208958093070277
:101AC00008958093080208958093090208950F9362
:101AD0001F93CF93DF938C01CB01C091F901D0917B
:101AE000FA0162E070E00E94C51210C0988129815D
:101AF0008A81823041F4E92FF22F858190E08017AE
:101B0000910709F460870F80D885C02D209771F761
:101B1000DF91CF911F910F9108959C01E091F90100
:101B2000F091FA0114C0A081B1818281843061F406
:101B3000848190E08217930739F4868190E08617BC
:101B4000970711F413964C930780F085E02D30979A
:101B500051F7089590939900809398000895BF924B
:101B6000CF92DF92EF92FF920F931F93CF93DF9369
:101B7000EC01F62ED42EC22EB02EE091F901F09198
:101B8000FA01309799F489E090E00E94EC12FC0190
:101B90009093FA018093F901D183C083F382108678
:101BA0001782D282C4820583E6821AC0CF010780E1
:101BB000F085E02D3097D1F78C0189E090E00E940C
:101BC000EC12FC01D80118969C938E931797D18341
:101BD000C083F382D282C482B582E68210861782E5
:101BE000DF91CF911F910F91FF90EF90DF90CF90F9
:101BF000BF900895EF92FF921F93CF93DF937C01E4
:101C0000C0919A00D0919B00209711F011E012C072
:101C100085E090E00E94EC12FC0190939B00809381
:101C20009A00F182E08212821482138210E012C0C4
:101C30001F5FEC018B819C810097D1F785E090E0DC
:101C40000E94EC12FC019C838B83F182E082128360
:101C500014821382812FDF91CF911F91FF90EF901B
:101C60000895EF92FF920F931F93CF93DF93E0912C
:101C70009A00F0919B0080E090E00380F481E02DD9
:101C800001963097D1F7880F991F0E94EC1280932C
:101C90009C0090939D00C0919A00D0919B0001C040
:101CA000EC01E880F9808A8190E0880F991F00910B
:101CB0009C0010919D00080F191FF701808190E092
:101CC0000E94EC12F8018083918320E030E016C07E
:101CD0008A8190E0880F991FE0919C00F0919D000F
:101CE000E80FF91F0190F081E02DE20FF31FD701FB
:101CF000A20FB31F8C9180832F5F3F4FF70180812C
:101D000090E02817390724F38B819C81009741F6D6
:101D1000DF91CF911F910F91FF90EF9008956F92F7
:101D20007F928F929F92AF92BF92CF92DF92EF926B
:101D3000FF920F931F93CF93DF93E091F901F091FE
:101D4000FA01CC24DD2409C08281823019F4089480
:101D5000C11CD11C0780F085E02D3097A9F7C60182
:101D6000880F991F0E94EC1280931602909317021D
:101D70000894C108D1085601AA0CBB1C0894C11CC8
:101D8000D11CC1E0D0E0882499244FC0E091F90132
:101D9000F091FA01A9E0EA2EF12C16C0A081B181E0
:101DA000848190E08C179D0719F48381E80EF11C63
:101DB00015968C9115978C1721F48281823009F445
:101DC0004D010780F085E02D309741F70091160214
:101DD000109117020A0D1B1DC7010E94EC12D801B9
:101DE0008C9311969C9320E030E0E0911602F091E4
:101DF0001702EA0DFB1D0190F081E02DE20FF31FA9
:101E0000D401A20FB31F8C9180832F5F3F4F2930E5
:101E1000310559F7E0911602F0911702EA0DFB1D0A
:101E20000190F081E02DE2822196CC16DD060CF0C7
:101E3000ADCFE1E0EE2EF12C79E0A72EB12C662497
:101E4000772488249924A5C0A091F901B091FA01C2
:101E500013C0ED91FC9111978181823049F4858105
:101E600090E08E159F0521F48481682E772406C0AA
:101E700017960D90BC91A02D109759F701E010E036
:101E80007DC04091F9015091FA0172C0DA01ED91E3
:101E9000FC9111978181843009F065C016968C9170
:101EA000169790E08017910709F05DC014968C9109
:101EB00090E08E159F0509F056C0DF019501BF0126
:101EC000675F7F4FE0911602F0911702E80DF91D50
:101ED0000190F081E02DE20FF31F8D9180832F5F41
:101EE0003F4FA617B70771F7E9E0F0E0AE0EBF1E4F
:101EF000A091F901B091FA0134C012968C91129719
:101F0000853059F514968C91149790E08E159F05A5
:101F100021F515968C91159790E080179107E9F4BB
:101F2000CD91DC9111979501BE01695F7F4FE091E2
:101F30001602F0911702E80DF91D0190F081E02DD5
:101F4000E20FF31F899180832F5F3F4FC617D7079A
:101F500071F787E090E0A80EB91E17960D90BC911E
:101F6000A02D109751F6DA0117964D915C911897B4
:101F70004115510509F08ACF0F5F1F4F601671069A
:101F80000CF07FCF0894E11CF11CE2E0F0E08E0E33
:101F90009F1ECE14DF040CF057CFDF91CF911F911D
:101FA0000F91FF90EF90DF90CF90BF90AF909F90F8
:101FB0008F907F906F900895AF92BF92CF92EF92E3
:101FC000FF920F931F93CF93DF93EC015B01122FCE
:101FD000E091F901F091FA0118C0A081B1818481EA
:101FE00090E0C817D90771F4868190E08A159B05A7
:101FF00049F48281843031F414968C9114978F5F68
:1020000014968C930780F085E02D309731F787E0A8
:1020100090E00E94EC12FC0187E0808385E08183E0
:1020200012830383F582E482C682CF0167E045E034
:102030002C2F0A2DEE240E94AF0DDF91CF911F911E
:102040000F91FF90EF90CF90BF90AF900895AF9217
:10205000BF92CF92DF92EF92FF920F9342305105E1
:1020600059F04330510569F04130510571F4B09297
:10207000F401A092F30109C0B092F601A092F5011B
:1020800004C0B092F801A092F70120583F4F0E947F
:10209000DC0F0F91FF90EF90DF90CF90BF90AF904B
:1020A0000895AF92BF92CF92DF92EF92FF920F937B
:1020B0004230510559F04330510569F04130510526
:1020C00071F4B0929300A092920009C0B092950072
:1020D000A092940004C0B0929700A09296000E9433
:1020E000DC0F0F91FF90EF90DF90CF90BF90AF90FB
:1020F0000895EF920F93CF93DF93082FE62EA091D0
:10210000F901B091FA01C0E0D0E014C0ED91FC916A
:1021100011978581801751F412968C911297823015
:1021200029F484818F5F8483C82FD0E017960D90A7
:10213000BC91A02D109751F789E090E00E94EC121D
:10214000FC0189E0808384E08183E282138214822F
:102150001582168217821086CF0169E044E0202F95
:1021600000E0EC2E0E94AF0DCE01DF91CF910F91D8
:10217000EF900895DF92EF92FF920F931F93CF930A
:10218000DF93E82E162FF42ED22EA091F901B091F4
:10219000FA01C0E0D0E014C0ED91FC911197858167
:1021A0008E1551F412968C911297823029F4848105
:1021B0008F5F8483C82FD0E017960D90BC91A02D1F
:1021C000109751F789E090E00E94EC12FC0189E041
:1021D000808384E08183128313821482F582D68205
:1021E00007831086CF0169E044E02E2D00E0EC2E3D
:1021F0000E94AF0DCE01DF91CF911F910F91FF9003
:10220000EF90DF900895EF920F931F9310911402B7
:102210001F5F1093140289E090E00E94EC12FC0111
:1022200089E0808389E090E09383828382E08183E8
:1022300014821583168280E887838AE18087CF0124
:1022400069E042E020E000E0EE240E94AF0D812F23
:1022500090E01F910F91EF9008950F931F93CF93EC
:10226000DF938C01FC0101900020E9F7E81BF90BDA
:10227000CF01880F991F0E94EC12EC01F801019028
:102280000020E9F7E01BF10BEE0FFF1FE88323E0CE
:102290002983AC0120E030E009C0F801E20FF31F10
:1022A0008081FA01808311822F5F3F4FF8010190F6
:1022B0000020E9F73197E01BF10B4E5F5F4F2E17BF
:1022C0003F0758F3CE010E94FA0D90E0DF91CF91C5
:1022D0001F910F9108950F931F93CF93DF938C015C
:1022E000EB01CA010E942D11282FE091F901F09114
:1022F000FA0114C0A081B1818281843061F48481AB
:1023000090E08017910739F4868190E08C179D0743
:1023100011F418962C930780F085E02D309751F733
:10232000DF91CF911F910F910895CF93DF93EC012F
:10233000CB010E942D11382FA091F901B091FA0123
:1023400015C09C9111962C91119712968C91129711
:10235000823041F4E92FF22F858190E08C179D07A0
:1023600009F4368317960D90BC91A02D109749F76C
:10237000DF91CF9108950E942D111816190614F4BB
:102380008093130208950E942D111816190614F453
:102390008093120208950E942D111816190614F444
:1023A0008093110208951F93CF93DF9386E00E94DC
:1023B000B50CC82F81FF02C00E94BC0AC4FF02C036
:1023C0000E941D0BC6FF02C00E94E70BC2FF02C0A5
:1023D0000E94EC0A87E00E94B50C182F87E060E0AD
:1023E0000E94E70C87E0612F0E94E70CDF91CF91FC
:1023F0001F9108950E948F0E0E94310E0E947B094A
:1024000080E061E00E94E70C80E00E94B50C80FD56
:10241000FBCF81E062E00E94E70C84E060E80E946C
:10242000E70C80E260E40E94E70C83E268E00E942F
:10243000E70C87E269E00E94E70C8DE06FE00E9404
:10244000E70C8BE06FE00E94E70C89E068ED0E94EA
:10245000E70C8FE061E30E94E70C87E066ED0E94E5
:10246000E70C85E062E00E94E70C80E06CEC0E94E3
:10247000E70C0895FC0111821082778366837583CF
:1024800064835383428353874287518740878FEF0A
:1024900084870895FC0120813181828193812817EE
:1024A00039071CF020E030E016C0A681B7816D939B
:1024B00082859385019721F482819381A81BB90BB2
:1024C00093878287B783A6838081918101969183C8
:1024D000808321E030E0C9010895FC018081918171
:1024E000892BE1F3A481B5812D9180859185019798
:1024F00021F482819381A81BB90BB583A4839187B2
:10250000808780819181019791838083822F0895B4
:10251000CF93DF93FC01EB0180819181181619069E
:102520001CF02FEF3FEF17C0A481B5812D9180855E
:102530009185019721F482819381A81BB90BB58302
:10254000A483918780878081918101979183808383
:10255000288321E030E0C901DF91CF910895DC9A12
:10256000F894E0918800F09189000995089520E0A1
:1025700030E040EA5FE005C0FA013197F1F72F5FE4
:102580003F4F28173907C4F3089597FB092E0726F4
:102590000AD077FD04D00CD006D000201AF4709534
:1025A00061957F4F0895F6F7909581959F4F089517
:1025B000AA1BBB1B51E107C0AA1FBB1FA617B70769
:1025C00010F0A61BB70B881F991F5A95A9F7809585
:1025D0009095BC01CD010895CF93DF93BC0182306B
:1025E000910510F462E070E0A0912802B0912902F8
:1025F000ED01E0E0F0E040E050E021C08881998109
:102600008617970769F48A819B81309719F0938325
:10261000828304C09093290280932802FE0134C073
:102620006817790738F44115510519F08417950793
:1026300008F4AC01FE018A819B819C01E90120978D
:10264000E9F641155105A9F1CA01861B970B0497BC
:1026500008F4BA01E0E0F0E02AC08D919C91119756
:1026600084179507F9F46417750781F412968D9114
:102670009C911397309719F09383828304C09093B1
:10268000290280932802FD0132964FC0CA01861BA1
:10269000970BFD01E80FF91F6193719302978D93DA
:1026A0009C9343C0FD01828193819C01D9011097C5
:1026B000A1F68091260290912702892B41F4809106
:1026C0008C0090918D009093270280932602409178
:1026D0008E0050918F004115510541F44DB75EB702
:1026E00080918A0090918B00481B590B2091260203
:1026F0003091270224173507B0F4CA01821B930BCF
:102700008617970780F0AB014E5F5F4F84179507E0
:1027100050F0420F531F5093270240932602F901B5
:102720006193719302C0E0E0F0E0CF01DF91CF91BF
:102730000895CF93DF93009709F450C0EC012297DE
:102740001B821A82A0912802B0912902109709F1E8
:1027500040E050E0AC17BD0708F1BB83AA83FE013F
:1027600021913191E20FF31FAE17BF0779F48D91DC
:102770009C911197280F391F2E5F3F4F3983288373
:1027800012968D919C9113979B838A8341155105D5
:1027900071F4D0932902C093280220C012968D9123
:1027A0009C911397AD01009711F0DC01D3CFFA0192
:1027B000D383C28321913191E20FF31FCE17DF073C
:1027C00069F488819981280F391F2E5F3F4FFA01E4
:1027D000318320838A819B8193838283DF91CF9190
:1027E0000895FB01DC0102C001900D924150504060
:1027F000D8F70895E199FECF9FBB8EBBE09A992749
:102800008DB30895262FE199FECF9FBB8EBB2DBBC4
:102810000FB6F894E29AE19A0FBE01960895F894E3
:02282000FFCFE8
:10282200422E5361757465720041565249535020CD
:102832006D6B3220424C3032380030303030413013
:102842003031323832353500007020002A02000063
:00000001FF
